:020000040000FA
:10000000A4EF07F0D9CFE5FFE1CFD9FF00C0E5FFAE
:1000100001C0E5FF02C0E5FF03C0E5FF04C0E5FF46
:1000200005C0E5FF06C0E5FF07C0E5FF08C0E5FF26
:1000300009C0E5FF0AC0E5FF0BC0E5FF0CC0E5FF06
:10004000020EDBCF00F0030EDBCF01F0040EDBCF9E
:1000500002F0050EDBCF03F0060EDBCF04F00050FC
:100060000110D8A4E3D002C0E9FF03C0F3FF04509D
:1000700069EC07F0056EF3CF06F0000E065C02E1B6
:100080000A0E055CD8B057D00DC0E5FF0EC0E5FFE5
:100090000E6A05340E36E8340E36FC0B0D6E000E7B
:1000A000FB6E000EFA6EBE0E0D260E50FA22D8B070
:1000B000FB2A0D50E4CF0EF0E4CF0DF0F96E73EF94
:1000C00000F077EF00F07BEF00F07FEF00F083EFC0
:1000D00000F087EF00F08BEF00F08FEF00F093EF70
:1000E00000F097EF00F0010E056E066A27D0020EB1
:1000F000056E066A23D0040E056E066A1FD0080E30
:10010000056E066A1BD0100E056E066A17D0200E0B
:10011000056E066A13D0400E056E066A0FD0800E7B
:10012000056E066A0BD0C00E056E066A07D0056A1A
:10013000010E066E03D0C00E056E066AB886065024
:10014000E56E0550E56E020EE56E580EE56E5AEC52
:1001500005F0076EF3CF08F0040EE126096A0A6A7B
:100160002D0E0826310E0922010E0A220650E56ED8
:100170000550E56E010EE56E2C0EE56E5AEC05F0AD
:10018000056EF3CF06F0040EE1260B6A0C6A0C50E4
:10019000E56E0B50E56E0650E56E0550E56E0A50B3
:1001A000E56E0950E56E0850E56E0750E56E5BECB4
:1001B00001F0056EF3CF06F0F4CF07F0E9CF08F0B9
:1001C000080EE126000EE56E000EE56E000EE56EEF
:1001D000040EE56E0850E56E0750E56E0650E56EBC
:1001E0000550E56E5BEC01F0056EF3CF06F0F4CF41
:1001F00007F0E9CF08F0080EE126FF0E0526FF0EF6
:100200000622FF0E0722FF0E08220650E56E05505B
:10021000E56E3C0EF6EC05F0020EE126AB8EAB88E7
:100220000D0E0DEC08F0F36A010E28D00050010A03
:1002300002E1015001E020D0040E0226000E03224C
:10024000000E042202C0E9FF03C0F3FF045093EC48
:1002500007F0026E025007E0949A94889496C76A59
:10026000210EC66E06D0949A94889486C76A250E8D
:10027000C66EF36A010E02D0F36AE86AE4CF0CF0AE
:10028000E4CF0BF0E4CF0AF0E4CF09F0E4CF08F0BC
:10029000E4CF07F0E4CF06F0E4CF05F0E4CF04F0BC
:1002A000E4CF03F0E4CF02F0E4CF01F0E4CF00F0BC
:1002B000E4CFD9FF1200D9CFE5FFE1CFD9FF00C0CD
:1002C000E5FF01C0E5FF02C0E5FF03C0E5FF04C094
:1002D000E5FF05C0E5FF06C0E5FF07C0E5FF08C074
:1002E000E5FF09C0E5FF0AC0E5FF0BC0E5FF0CC054
:1002F000E5FF0DC0E5FF020EDBCF00F0030EDBCF04
:1003000001F0040EDBCF02F0050EDBCF03F0060E8A
:10031000DBCF04F0070EDBCF05F0080EDBCF06F0D5
:10032000090EDBCF07F0D88003AED890086A0836F4
:1003300008500FE0031C0C6E021C0B6E011C0A6EB1
:10034000001C096E092A0DE10A2A0BE10B4A0C2A4E
:1003500008D000C009F001C00AF002C00BF003C0D1
:100360000CF009C000F00AC001F00BC002F00CC094
:1003700003F0D88007AED890096A093609500FE01B
:10038000071C0D6E061C0C6E051C0B6E041C0A6E01
:100390000A2A0DE10B2A0BE10C4A0D2A08D004C0F1
:1003A0000AF005C00BF006C00CF007C00DF00D50B0
:1003B000E56E0C50E56E0B50E56E0A50E56E03508D
:1003C000E56E0250E56E0150E56E0050E56E32ECD0
:1003D00002F0006EF3CF01F0F4CF02F0E9CF03F0AA
:1003E000080EE1260950081A085016E0031C076E93
:1003F000021C066E011C056E001C046E042A04E13A
:10040000052A02E1064A072A07C0E9FF06C0F4FFF1
:1004100005C0F3FF045007D003C0E9FF02C0F4FF9A
:1004200001C0F3FF0050E4CF0DF0E4CF0CF0E4CFB7
:100430000BF0E4CF0AF0E4CF09F0E4CF08F0E4CF0A
:1004400007F0E4CF06F0E4CF05F0E4CF04F0E4CF0A
:1004500003F0E4CF02F0E4CF01F0E4CF00F0E4CF0A
:10046000D9FF1200D9CFE5FFE1CFD9FF00C0E5FFEA
:1004700001C0E5FF02C0E5FF03C0E5FF04C0E5FFE2
:1004800005C0E5FF06C0E5FF07C0E5FF08C0E5FFC2
:1004900009C0E5FF0AC0E5FF0BC0E5FF0CC0E5FFA2
:1004A0000DC0E5FF020EDBCF00F0030EDBCF01F045
:1004B000040EDBCF02F0050EDBCF03F0060EDBCF20
:1004C00004F0070EDBCF05F0080EDBCF06F0090EB7
:1004D000DBCF07F0086A096A0A6A0B6A200E0C6E05
:1004E0000344010B0D6E010E0D160050002601365F
:1004F000023603360850082609360A360B360D50E8
:10050000D8A4088007500B5C08E106500A5C05E19E
:100510000550095C02E10450085C09E30450085EE0
:100520000550095A06500A5A07500B5A00800C2EE3
:10053000D7D703C0E9FF02C0F4FF01C0F3FF0050AA
:10054000E4CF0DF0E4CF0CF0E4CF0BF0E4CF0AF0F1
:10055000E4CF09F0E4CF08F0E4CF07F0E4CF06F0F1
:10056000E4CF05F0E4CF04F0E4CF03F0E4CF02F0F1
:10057000E4CF01F0E4CF00F0E4CFD9FF1200D9CFEF
:10058000E5FFE1CFD9FF00C0E5FF01C0E5FF02C0F4
:10059000E5FF03C0E5FF04C0E5FF05C0E5FF06C0B9
:1005A000E5FF07C0E5FF08C0E5FF09C0E5FF0AC099
:1005B000E5FF0BC0E5FF020EDBCF00F0030EDBCF43
:1005C00001F0040EDBCF02F0050EDBCF03F0060EC8
:1005D000DBCF04F0070EDBCF05F0080EDBCF06F013
:1005E0000050011006E00050010A02E1015001E054
:1005F0002DD0076A086A0850800FF36E0650800FEE
:10060000F35C02E10550075C21E207500224096E09
:10061000085003200A6EE86A08BEE86804200B6EE2
:1006200009C0E9FF0AC0F3FF0B5093EC07F0096E15
:100630000950E56E0150E56E0050E56E39EC06F0AC
:10064000030EE126072AD8B0082AD5D7E4CF0BF04D
:10065000E4CF0AF0E4CF09F0E4CF08F0E4CF07F0EC
:10066000E4CF06F0E4CF05F0E4CF04F0E4CF03F0EC
:10067000E4CF02F0E4CF01F0E4CF00F0E4CFD9FF03
:100680001200D9CFE5FFE1CFD9FF00C0E5FF01C0DF
:10069000E5FF02C0E5FF03C0E5FF04C0E5FF020E71
:1006A000DBCF00F0030EDBCF01F0000E015C02E1B6
:1006B000080E005C11E2010E026E036A005006E0B3
:1006C000E86CD89002360336010FFCE3FF0E021AE5
:1006D0008950021602C089FF000E015C02E1080E7B
:1006E000005C1AE3000E015C02E1100E005C14E2F3
:1006F0000050036EF80E0326010E046E035005E051
:10070000E86CD8900436010FFDE3041C036E03501F
:100710008A14026E02C08AFF000E015C02E1100E14
:10072000005C15E3000E015C02E1180E005C0FE2B4
:10073000F00E0026010E016E005005E0E86CD89026
:100740000136010FFDE3011C006E00508B16E4CF53
:1007500004F0E4CF03F0E4CF02F0E4CF01F0E4CF03
:1007600000F0E4CFD9FF1200D9CFE5FFE1CFD9FFE8
:1007700000C0E5FF01C0E5FF02C0E5FF03C0E5FFE3
:10078000020EDBCF00F0030EDBCF01F0000E015CA8
:1007900002E1080E005C0DE2010E026E036A0050D9
:1007A00006E0E86CD89002360336010FFCE30250F5
:1007B0009212000E015C02E1080E005CD870026A21
:1007C00002360250D880E866D890026A023602509B
:1007D000800F700F0FE20050026EF80E0226010E1D
:1007E000036E025005E0E86CD8900336010FFDE37C
:1007F00003509312000E015C02E1100E005CD870F1
:10080000026A02360250D880E866D890026A023640
:100810000250800F680F0DE2F00E0026010E016EEF
:10082000005005E0E86CD8900136010FFDE301505F
:100830009412E4CF03F0E4CF02F0E4CF01F0E4CF70
:1008400000F0E4CFD9FF1200D9CFE5FFE1CFD9FF07
:1008500000C0E5FF01C0E5FF02C0E5FF03C0E5FF02
:10086000020EDBCF00F0030EDBCF01F0000E015CC7
:1008700002E1080E005C0DE2010E026E036A0050F8
:1008800006E0E86CD89002360336010FFCE3025014
:10089000891A000E015C02E1080E005CD870026A41
:1008A00002360250D880E866D890026A02360250BA
:1008B000800F700F0FE20050026EF80E0226010E3C
:1008C000036E025005E0E86CD8900336010FFDE39B
:1008D00003508A1A000E015C02E1100E005CD87011
:1008E000026A02360250D880E866D890026A023660
:1008F0000250800F680F0DE2F00E0026010E016E0F
:10090000005005E0E86CD8900136010FFDE301507E
:100910008B1AE4CF03F0E4CF02F0E4CF01F0E4CF90
:1009200000F0E4CFD9FF1200D9CFE5FFE1CFD9FF26
:1009300000C0E5FF01C0E5FF02C0E5FF03C0E5FF21
:1009400004C0E5FF020EDBCF00F0030EDBCF01F0A9
:10095000000E015C02E1080E005C0FE2010E026E67
:10096000036A005006E0E86CD89002360336010FA7
:10097000FCE38950021202C089FF000E015C02E113
:10098000080E005C18E3000E015C02E1100E005C32
:1009900012E20050036EF80E0326010E046E03509F
:1009A00005E0E86CD8900436010FFDE304508A108E
:1009B000026E02C08AFF000E015C02E1100E005CB4
:1009C00013E3000E015C02E1180E005C0DE2F00E74
:1009D0000026010E016E005005E0E86CD89001364B
:1009E000010FFDE301508B12E4CF04F0E4CF03F0DC
:1009F000E4CF02F0E4CF01F0E4CF00F0E4CFD9FF80
:100A00001200006A016A080E0001606F0001616B4C
:100A1000010E0001636F000E036E600E026E800E09
:100A2000046E0450E56E0350E56E0250E56E000E54
:100A3000E56E000EE56E02EC00F0050EE126FC0E00
:100A4000E56ED8EC07F0E12A002AD8B0012A01505F
:100A5000800F460F02E1990E005C11E3000EE56E77
:100A6000080EE56E41EC03F0020EE126000EE56E85
:100A7000090EE56E41EC03F0020EE12610D0000EE7
:100A8000E56E080EE56E94EC04F0020EE126000E11
:100A9000E56E090EE56E94EC04F0020EE1260050BE
:100AA000300A03E10150750A01E0CED7006A016AFD
:100AB000CBD71200D9CFE5FFE1CFD9FF00C0E5FFCA
:100AC00001C0E5FF02C0E5FF03C0E5FF020EDBCF7A
:100AD00000F0030EDBCF01F0040EDBCF02F0050EB9
:100AE000DBCF03F000500001666F0150676F0250CA
:100AF0000001686F0350696F0001665100016803CF
:100B0000F3CF00F0F4CF01F0005000016A6F015004
:100B10006B6F0001665100016903F3CF00F0000123
:100B2000675100016803F3CF01F001500026000176
:100B30006B51002600506B6F6BC0F3FF6A51E4CF1E
:100B400003F0E4CF02F0E4CF01F0E4CF00F0E4CF13
:100B5000D9FF1200380EF66E100EF76E000EF86E0A
:100B60000900F550056E0900F550066E055002E1CA
:100B700006503BE00900F550006E0900F550016E8B
:100B80000900F550026E09000900F550E96E0900F0
:100B9000F550EA6E090009000900F550036E0900DE
:100BA000F550046E09000900F6CF07F0F7CF08F002
:100BB000F8CF09F000C0F6FF01C0F7FF02C0F8FF50
:100BC000035002E1045007E00900F550EE6E030601
:100BD000F8E20406F9D707C0F6FF08C0F7FF09C01E
:100BE000F8FF0506C4E20606C5D71200D9CFE5FF17
:100BF000E1CFD9FF00C0E5FF01C0E5FF02C0E5FF7E
:100C0000006E020EDBCF01F0030EDBCF02F0AC6A08
:100C1000AB6A00B0AC8800A202D0AC8CAB8C00A454
:100C200001D0AC8E00A602D0AB8801D0AB8A00A860
:100C300002D0AC8401D0AC949E9800AC02D09D8AC6
:100C400001D09D9A9E9A00AE02D09D8801D09D98B9
:100C50000250B06E0150AF6E949C948EAC8AAB8EF5
:100C6000E4CF02F0E4CF01F0E4CF00F0E4CFD9FF0D
:100C70001200D9CFE5FFE1CFD9FF00C0E5FF01C0E9
:100C8000E5FF02C0E5FF03C0E5FF020EDBCF00F089
:100C9000030EDBCF01F0040EDBCF02F00050011099
:100CA00008E102500DEC08F023EC08F0036E03504D
:100CB000FBE10050010A02E1015001E002D002C054
:100CC000C9FFE4CF03F0E4CF02F0E4CF01F0E4CFBA
:100CD00000F0E4CFD9FF1200D9CFE5FFE1CFD9FF73
:100CE00000C0E5FF01C0E5FF020EDBCF00F0030E00
:100CF000DBCF01F0005007E00050080A0AE0005086
:100D0000100A0DE011D00150E56EC4EC07F0E12AA5
:100D10000BD00150E56EBAEC07F0E12A05D0015086
:100D2000E56EB0EC07F0E12AE4CF01F0E4CF00F08B
:100D3000E4CFD9FF1200D9CFE5FFE1CFD9FF00C042
:100D4000E5FF01C0E5FF020EDBCF00F0030EDBCFB5
:100D500001F0005007E00050080A0AE00050100AB5
:100D60000DE011D00150E56EE2EC07F0E12A0BD066
:100D70000150E56ED8EC07F0E12A05D00150E56E90
:100D8000CEEC07F0E12AE4CF01F0E4CF00F0E4CFAD
:100D9000D9FF1200D9CFE5FFE1CFD9FF00C0E5FFB1
:100DA00001C0E5FF02C0E5FF020EDBCF00F0030E3D
:100DB000DBCF01F00050011006E19E9A7FEC07F0B6
:100DC000026E02500BD00050010A02E1015001E016
:100DD00004D0C7A002D0C95001D0E86AE4CF02F025
:100DE000E4CF01F0E4CF00F0E4CFD9FF1200D9CF77
:100DF000E5FFE1CFD9FF00C0E5FF01C0E5FF020E2E
:100E0000DBCF00F0030EDBCF01F00050011006E154
:100E10009EAA02D0010E0FD0E86A0DD00050010A40
:100E200002E1015001E006D0C7A002D0010E03D0BC
:100E3000E86A01D0E86AE4CF01F0E4CF00F0E4CF43
:100E4000D9FF1200D9CFE5FFE1CFD9FF00C0E5FF00
:100E5000020EDBCF00F0005007E00050080A09E066
:100E60000050100A0BE00ED005EC08F0006E0050A8
:100E700009D0FDEC07F0006E005004D0F5EC07F04F
:100E8000006E0050E4CF00F0E4CFD9FF1200D9CFBC
:100E9000E5FFE1CFD9FF00C0E5FF01C0E5FF020E8D
:100EA000DBCF00F0030EDBCF01F00050011009E1B1
:100EB00023EC08F0006E005002E0E86A03D0010E57
:100EC00001D0E86AE4CF01F0E4CF00F0E4CFD9FF2D
:100ED0001200E8AE06D0F3CFEAFFEE50EECFF3FFFC
:100EE0001200E8BC0BD0E9CFF6FFF3CFF7FFF86EA6
:100EF0000900F5500900F5CFF3FF12001200F00EC3
:100F000000016D156D6FABAC04D06D91ABA001D03D
:100F10006D81ABA402D000016D85ABA202D00001AF
:100F20006D87AE501200E8AE04D0F3CFEAFFEE506A
:100F30001200E8BC08D0E9CFF6FFF3CFF7FFF86E58
:100F40000900F5501200120017EEFFF027EEFFF037
:100F5000F86AA68EA69CAAEC05F001EC05F0FFD776
:100F6000D9CFE5FFE1CFD9FF020EDBCF8BFFE4CF76
:100F7000D9FF1200D9CFE5FFE1CFD9FF020EDBCFB9
:100F80008AFFE4CFD9FF1200D9CFE5FFE1CFD9FF27
:100F9000020EDBCF89FFE4CFD9FF1200D9CFE5FFE6
:100FA000E1CFD9FF020EDBCF94FFE4CFD9FF1200CF
:100FB000D9CFE5FFE1CFD9FF020EDBCF93FFE4CF1E
:100FC000D9FF1200D9CFE5FFE1CFD9FF020EDBCF69
:100FD00092FFE4CFD9FF1200D9CFE5FFE1CFD9FFCF
:100FE000F36AE86AE4CFD9FF1200D9CFE5FFE1CF79
:100FF000D9FF8250E4CFD9FF1200D9CFE5FFE1CF6E
:10100000D9FF8150E4CFD9FF1200D9CFE5FFE1CF5E
:10101000D9FF8050E4CFD9FF1200ACAC04D0AC9023
:1010200000016DB3AC80AD6E1200D9CFE5FFE1CF0A
:10103000D9FFE4CFD9FF120001004E1000006C0070
:10104000000001000000000EACA2010F1200000021
:020000040030CA
:0E000000FFF2FFFEFFFFBBFFFFFFFFFFFFFF52
:00000001FF
